:020000040000FA
:100000000000831203139F01831607309C00063003
:100010009F00FF308600E0308500F03087008312BB
:1000200085018701061C2028851A142810308500B8
:10003000851A18280130870006181C2885018701B9
:10004000861C2E28851A222810308500851A26281D
:100050000230870086182A2885018701061D3C2862
:10006000851A302810308500851A3428043087001E
:100070000619382885018701861D4A28851A3E28D9
:1000800010308500851A42280830870086194628D6
:1000900085018701061E5828851A4C2810308500D6
:1000A000851A502811308500061A542885018701C9
:1000B000861E6628851A5A2810308500851A5E2803
:1000C00012308500861A622885018701061F742870
:1000D000851A682810308500851A6C281430850030
:1000E000061B702885018701861F1228851A76282D
:1000F00010308500851A7A2818308500861B7E28E6
:06010000850187011228B1
:04010600003400348D
:02400E00323F3F
:00000001FF
